:0300000002194B97
:0C194B0078FFE4F6D8FD7581C20200367A
:0100110022CC
:06167A008B308A31893239
:10168000756A027F481217F7121997EF20E0F9AB3D
:1016900030AA31A93212068D7872E6FE08E6FDED19
:0116A000FF4A
:0116A1002226
:100EBD0043525354005341564500434647002D3E7F
:100ECD0053320052415445434C5220554E495442E1
:100EDD004C4E4B545249475452455644464C54532C
:100EED0041564552535420535720202E3235203130
:100EFD00732020327320203573202031307320333E
:100F0D00307320316D2020326D2020356D20203141
:100F1D00306D2033306D2031682020326820203430
:100F2D0068202000000001000400080014002800C3
:100F3D007800F001E004B009601C2038407080E1B9
:100F4D000046656574596172644D6574724F6666CD
:0D0F5D00204F6E20204E6F2020596573201C
:1017480025E02430F582E4340FF583220532E532B2
:0E175800C394022275F004A4245AF9740F22DF
:1015250078B576AB0876CD087600087604E408F63B
:1015350008760108F60876FA08764008F608F608EF
:10154500F608F67BFF7A0E79BD1215C17F051214D8
:04155500BA0216249C
:10181200756E1D756FC01214F078B6E664CD700453
:0918220018E664AB600312152501
:01182B00229A
:0D191300C2AF7DC07C1DE4FF12189FD2AF53
:0119200022A4
:1014F000753FFF856E40856F4175420075430075ED
:1015000044B5E4FFAB3FAA40A9418F827583001226
:101510000660AB42AA43A9448F8275830012069FDE
:041520000FBF0EE00B
:0115240022A4
:101624007D01E4FF1217667BFF7A0E79C21215C1A1
:10163400121913C2AF7FB57B0E7DC07C1D1218A991
:0D164400D2AF7F021214BAE4FDFF02176658
:100A3700E4F5307BFF7A0E79C71215C17F051214D2
:100A4700BAA297829650FAA296920FA2979210E5B1
:100A57003075F004A424D0F9740E35F0FA7BFF1238
:100A670015C17F051214BA853031E4F5327BFF7A60
:100A77000E79CB1215C1E53024FE602E14603314B5
:100A870060341460392405703D7F01EF12174878F0
:100A9700B7E6FC08E6FD7401936D7003E4936C7090
:100AA700028F320FBF0FE4020B4478B9E6F532022A
:100AB7000B6978BA800278C2E6F532020B8278C1F8
:100AC700E6F532020BA8E53065317083A20F309648
:100AD70001B35013A296920F30960C0530E530C340
:100AE70094094003E4F530A210309701B350D7A220
:100AF7009792103097D0E530B4090050C9900B0B8E
:100B0700F8282873020B26020B51020B57020B74AD
:100B1700020B87020B9A020BBC020BC2020BC80521
:100B270032E532C3940F4003753201E5321217489C
:100B3700E493FF74019378B7CFF608EFF6E53275C3
:100B4700F004A424F4F9740E8060121178020ACD1F
:100B57000532E532C394034003E4F53278B9A6328F
:100B6700E53275F004A4244EF9740F803D12175432
:100B77004003E4F53278BAA632E53212175C802AD0
:100B87001217544003E4F53278C2A632E532121741
:100B97005C80171217544003E4F53278C1A632E59A
:100BA7003275F004A42462F9740F35F0FA7BFF1252
:100BB70015C1020ACD121525020ACD121624020A02
:070BC700CD43A208020ACD94
:0A1963004552415300444F4E450029
:1017A200E4D3FCFD7B80FAF9F80207EC78B7E6F5A2
:0D17B2005608E6F55722E563AE6278062280
:10105900C20DC20EE4F531F532AE31AF321217A22C
:10106900401CE53064816016AF32AE311215F312BF
:10107900188B8F300532E53270DF053180DBE530C2
:10108900B48108E532153270021531AE31AF32E460
:10109900C31217A4700CD20D12192FE4F562F5636F
:1010A9008007853162853263E4F564F5657555809D
:0310B9001217AE5D
:0110BC002211
:0415F3008F828E83D2
:1015F7001217A24027E582AE837806C333CE33CED7
:10160700D8F9FD756A02EE7872F6CFEDCFEF08F6DE
:0C1617007F5012185F121997EF20E0F9C5
:0116230022A4
:03182C00CDEFCD30
:10182F00756A02EE7872F6ED08F67F5012185F12A5
:06183F001997EF20E0F90B
:011845002280
:10188B00756A017F501217F7121997EF20E0F9785C
:03189B0072E6FFF3
:01189E002227
:1018760012182CE4FFFE0FBF00010EBE0FF8BFA02A
:04188600F512188BB4
:01188A00223B
:06155900CBEFCBCAEECA85
:10155F00300D03300E27756A03EA7872F6EB08F642
:10156F0008EDF67F5012185F121997EF20E0F9E49B
:0D157F00FFFE0FBF00010EBE0FF8BFA0F56C
:01158C00223C
:10138A00753300753400753555E4F5321217B8C354
:10139A0033CE33CED8F97C002532FFEC3EFEAB3398
:1013AA00AA34A935853282758300120660FD1215AA
:1013BA00590532E532C3940640D275640075650654
:0113CA002200
:100F6A008E308F311217B8C333CE33CED8F92565F8
:100F7A00FFE5643EFEEEC0E0EFC0E0E530FDD0E004
:100F8A00FFD0E0FE1215590565E565700205641289
:100F9A0017B8C333CE33CED8F92565FFE5643EFED4
:100FAA00AD311215590565E565700205640559E507
:100FBA005970020558C3E5659440E56494004017EA
:100FCA00E4F564F5650563E56370020562AE62FFE8
:080FDA001217A25002D20D22F1
:10117800E4F564F5657BFF7A1979631215C1D20E1F
:10118800E4F53FF540AE3FAF401217A24021E540DD
:10119800AE3F7806C333CE33CED8F9F5658E647D7D
:1011A80081FF1215590540E54070DA053F80D6C227
:1011B8000E7BFF7A1979681215C1E4F562F563F5BB
:0511C80064F565C20D95
:0111CD0022FF
:10112100E4F53FF540F541F542AE41AF421217A259
:101131004044E5406481603EAF42AE411215F31276
:10114100188B8F40E54064807022AF3F053FFCFD66
:10115100FEFBFAF9120BCE7F2C12000EAE41AF420C
:10116100E4FCFDFBFAF9120BCE1219800542E542AF
:0611710070B7054180B3D8
:011177002255
:0212BD008F3F61
:1012BF00E4F540F541F542F543AE42AF431217A2B4
:1012CF004030E5416481602AAF43AE421215F312FC
:1012DF00188B8F41E541B4800FE540653F7007AF34
:1012EF0043AE420215F305400543E54370CB05427B
:0212FF0080C7A6
:0113010022C9
:1017DC001217AE78C2E6F55AE4F558F55912138A89
:0B17EC008562668563677F010210BD07
:10148200856230856331E565456460080531E53183
:101492007002053085666285676312138A85306241
:1014A200853163AE30AF311217A25007E4F562F511
:0814B20063D20D7F020210BDA0
:10189F00740478FF769612FF0322740078FF769611
:0418AF0012FF0322FF
:03003300020DF7C4
:0D0DF700C0E0C0F0C083C082C0D075D0083D
:100E0400E5D954F8FF1208650E31080E31100E4072
:100E1400180E5B200E42280E5B300E5D380E6340C8
:100E24000E5B480E7C500E995800000EA7856DDAB3
:100E3400C2DDC2DC756B00756C008070800EE56AE3
:100E440070028056056CE56C7002056B1200268FEB
:100E5400DAC2DDC2DC80558016D2DDC2DC804DC230
:100E6400DDC2DCE56A7004C2DA8041D2DA803DC2B8
:100E7400DDD2DC7568048034AFDA121957056CE5ED
:100E84006C7002056BC2DDC2DCE56A7004C2DA80F4
:100E94001BD2DA8017AFDA121957C2DDD2DC7568BB
:0E0EA400028009756804C2DDC2DCD2DAC2DB4E
:0B0EB200D0D0D082D083D0F0D0E0324E
:1016510043910C43920CE4F5DBEF25E0F5DB300F11
:101661000343DB0175DD2575DC2575D84453F8FE90
:0916710053F7FEE4F568D2E8220B
:10185F00E56830E002FF22E4F569756803EF25E0E3
:07186F00F56DD2DD7F0222BE
:1017F700E56830E002FF22E4F569156A756805EFD0
:0B18070025E04401F56DD2DD7F0222D8
:0619970020DBFDAF682219
:0D002600156AAF69056974722FF8E6FF22B4
:0C19570074722569F8EFF60569156A2224
:0E192100E4F5847585FFF592F5A475A5FF2207
:07198900EE3395E0FDFC22A6
:1016A200C20AC20CC209D2A2C2A0C2A1E4FDFF12A8
:1016B2001766E4FD7F011217667F081210BD7F04D2
:0316C2000210BD56
:10176600EF146011047016BD0104C2A78002D2A74F
:0E177600A2A7920B22BD0103C2A622D2A62278
:1010BD00EF14B40800505C9010D275F003A4C583F2
:1010CD0025F0C583730210EA0210F00210F7021129
:1010DD000302110502110302110F021117D20A7535
:1010ED00190122C20AA20B92A722D20C751A057DF4
:1010FD00017F010217668005C209C28722C209D28B
:10110D008722D209D28775180122C2A47F01121439
:04111D00BAD2A4227C
:10140A00300A12D5190F30A707C2A775191E800511
:10141A00D2A7751946E51AD39400400CD51A09C209
:10142A000CE4FD7F01121766300911D5180E3087BA
:0D143A0006C28775180522D28775181E227C
:10170800C374039FFE1392A0EEA2E192A1AF80CF13
:0F1718005480CFED547FCF4FCF8F80C2A2D2A28B
:01172700229F
:0615C1008B418A428943C0
:1015C700E4FCCFECCF7D201217080CBC04F4E4FC3C
:1015D700AB41AA42A9438C82758300120660FD6065
:0B15E7000ACFECCF1217080CBC04E583
:0115F20022D6
:040FE2008F828E83E9
:100FE600121989E47B0F7A27F9F8C31207EC50032C
:100FF60090270FAF82AE831219897B197AFC79FF8D
:1010060078FFD31207EC400390FC19E4F530741B0B
:101016002530F8E4F60530E530B405F2AE83AF824C
:101026001219897B007A00791B120BCEE51E701A05
:10103600753003741A2530F8E6FF741B2530F8C6A0
:10104600EFC6D530EE751B2080E27B007A00791B57
:031056000215C1BF
:1017840046554C4C0050524F47005A4C4F47004D61
:0E1794004F44310076312E39005472696700DF
:030013000216E7EB
:1016E700C0E0C0D075D01020060CAF8DEFAD8BF5E4
:1016F7005BEDF55CD206758D00758B00D0D0D0E020
:0117070032AF
:0214BA008F4061
:1014BC00E4F541F542C3E5429540E54194005023E3
:1014CC00900000AF82AE83E4FCFD7B207A4EF9F8ED
:1014DC00D31207EC4003A380EA0542E54270D6051F
:0314EC004180D26A
:0114EF0022DA
:0E192F007BFF7A1779841215C17F0A0214BA61
:1000360012192112196D1216A27F041214BA2097F2
:10004600127BFF7A1779891215C17F01121302D22A
:10005600AF80FE2096091203D8121059120A377A79
:1000660017798E1203CD7A1779931203CD7BFF7A17
:100076001779981215C17F041214BAE4FF121302FD
:100086001203D87F011214BA121059120011C212AB
:100096001214477F011214BAE4F55DF55E120012E0
:1000A600A2969200A2979201E4F52378A912084C31
:1000B60000000000E4F52478B112084CFFFFD8F1E7
:1000C60078A512084C00000000E4F55478AD12083B
:1000D6004C00000000C205C203C204E4F560F561ED
:1000E600F525F526F55BF55CC206F55FC20730120D
:1000F600FDC212300433A200309601B3400BA201B8
:10010600309701B340030201EA30961230970FC2CE
:1001160004E4F560F5617F041210BDE4F554A2967F
:100126009200A29792010201EA209605209702D238
:100136000830965D30975A300838C20878A51208FC
:1001460027EC4D4E4F78B1701312084C000000009A
:1001560078AD12082778A5120840801012084C00C6
:1001660000000078A512084C00000000D201D20061
:10017600802478BAE6601F0561E56170020560D3E8
:1001860094B8E560940B400ED2047F051210BD8032
:1001960005E4F560F561A200309601B3501DA29604
:1001A6009200309616200813E5546007E4F5547F54
:1001B6000680057554017F071210BDA20130970114
:1001C600B35021A297920130971A200817B2033034
:1001D600030F300D0712192FC20380081217DC8097
:1001E600031214821203E5200603020284C2AFC280
:1001F60006D2AFE4855C2F855B2EF52DF52CAF2F4F
:10020600AE2EAD2DAC2C7B107A27F9F81206C18FD5
:100216002F8E2E8D2D8C2CE4FB7A90F9F812134636
:100226008F2F8E2E8D2D8C2C78C1E66009C374B865
:100236009FFF740B9EFEE55F14601624FE6020246B
:10024600037038C3EF94B0EE9404500E755F0180CE
:1002560009D3EF9414EE94054024755F03801FC301
:10026600EF94B0EE94045016755F01300302D20786
:100276007BFF7A17799D1215C18003E4F55F05248B
:10028600E524C3940550030203C7E4F524FB7A0072
:10029600792712167A8E288F29E5276402600302D1
:1002A60003C778A9120833E8C0E0E9C0E0EAC0E075
:1002B600EBC0E078B9E6FDAF29AE28121271D0E0A6
:1002C600FBD0E0FAD0E0F9D0E0F8EB2FFFEA3EFEF3
:1002D600E93DFDE83CFC78A91208400523E523C367
:1002E600940550030203C778A9120827E47B05FA90
:1002F600F9F812134678A912084078A91208277847
:10030600A5120833C3EF9BFFEE9AFEED99FDEC981C
:10031600FC78A912084078B112082778A912083388
:10032600D31207EC400A78A912082778B1120840C0
:10033600E554600A78B3E6FE08E68E2AF52B78AB1C
:10034600E6FE08E68E28F529E5546006AF2BAE2AB0
:100356008004AF29AE28120FE230034F0526E526AA
:1003660070020525C378B896E5251896403DE4F554
:1003760025F5267F031210BD30050DE528FF120076
:100386000EAF29E52912000E200D1B78C2E6600D7E
:10039600300707432901C20780035329FEAF29AE60
:1003A60028120F6A800512192FC20378A91208278E
:1003B60078AD12084078A912084C00000000E4F558
:0703C6002312140A0200F4E7
:1003CD007BFF1215C17F041214BA22D2AF1218127C
:0803DD00C20F7F7012165122BD
:1016C500444C0021536967005A4C4F47004D4F4425
:1016D5003100312E390041707220303720323030E0
:0216E5003400CF
:10122000AF38AE37AD36AC35EC4D4E4F22EF24FF24
:10123000F538EE34FFF537ED34FFF536EC34FFF5D5
:101240003522E475382075374EF536F53522E475CC
:101250003801F537F536F53522FDFCAB38AA37A94C
:1012600036A835C30208027532007533007534B5EF
:01127000225B
:1003E50012193DEF70030206107F041210BDE4F5EB
:1003F50054C204F560F5611217BFEF1208650604D3
:1004050024060D2A056252042B6104996304EC65E8
:1004150005376C053D72053A7305667405D9760591
:10042500D178000006107BFF7A1679C51215C11226
:10043500124212193DEF700A121220600512122D98
:1004450080F012122070030206101217BF8F3112AE
:1004550012BDE4F538121252E47F06FE121259500D
:100465000A12188B8F3112061180ED12188B8F31FD
:10047500E53164806016E5316481601012000E126A
:10048500188B8F3112000E7530018003E4F530E5CD
:100495003070D82212126712124EF53112122060F6
:1004A5002412124212193DEF700A12122060051231
:1004B500122D80F0121220600312062A0531E53153
:1004C500C3940E40D7121220601A78B5B6AB070850
:1004D500B6CD0302060A7BFF7A1679C81215C17FCD
:1004E5000A0214BA0205CEE4FFFE12182CE4F53810
:1004F500121252E4FF7E08121259503312188B8FD4
:1005050030E538540FFFE4FEFDFCFBFAF9F8C312A1
:100515000802700F121980AE37AF381219027F200A
:1005250012000EAF301218467F2012061180C40249
:100535000601B20522021121121267E4F531AB3230
:100545000534E534AA337002053314F9120647FF62
:1005550012000E0531E531C3940E40E22243A20894
:100565002275320075330075347012124EF5311252
:100575001220602412124212193DEF700A12122045
:10058500600512122D80F0121220600312062A0552
:1005950031E531C3940240D7121220602CAE70AF02
:1005A50071EE3395E0FDFC78AD120833C3EF9BF592
:1005B5003CEE9AF53BED99F53AEC98F539AF3C7878
:1005C500BFE53BF608EFF6803C0214F07F041210FD
:1005D500BD0211787A1679CD12063E7A1679D212B5
:1005E500063E7F7612000E7BFF7A1679D71218EF3A
:1005F5001219807BFF7A1679DB1218EF021980E455
:0B06050078BFF608F602162412152537
:100610002212000EE5382401F538E43537F537E4C9
:100620003536F536E43535F535221217BFAB32AA2B
:1006300033A934853182758300EF12069F227BFF38
:070640001218EF12198022CD
:0A196D00E4F5955396BF53A27F22C4
:101447005389F0438901538FFE758C70E4F58A53F5
:10145700B8FD53B7FDD2A9D28C53890F4389905356
:101467008FEFF58DF58B4391105392EF53B8F753E8
:0B147700B7F7D2ABD28ED28AD2AA22E5
:03000B0002197760
:09197700D212758C70758A0032E1
:03001B0002199037
:07199000758D00758B00321C
:1018B3000D0A00303132333435363738394142433B
:0418C3004445460052
:1018C700AF53AB47AA48A949055322AF46AE45AD2A
:0418D70044AC4322B8
:101302005387BF75985053877FE4F5BABF010543F1
:10131200A240800353A2BFE4F5BD75BE30F5BF7590
:10132200BD035391FE4392014391025392FDC213B6
:1013320053B8EF53B7EF43B81078A3F618F678A472
:04134200F6D2AC2211
:0300230002158D36
:10158D00C0E0C0D075D01030981E78A3E6C3940F7C
:10159D00501418E6062492F8A69978A30618E6C307
:1015AD00941040027600C298309904C299C213D0AB
:0415BD00D0D0E03278
:080003002013FDD2138F992296
:1017280078A3E6D39400401508E6062492F8E6FF6D
:0F17380078A31608E6C394104005E4F6227F005C
:01174700227F
:03000E00020003EA
:1017BF007F207E4E78A3E67010D3EF9400EE940056
:0C17CF004007EF1F70EE1E80EB12172881
:0117DB0022EB
:1018EF00120647FF600C12000E740129F9E43AFA50
:0318FF0080EE2256
:0E193D0078A3E6D3940040037F01227F0022AE
:10184600CEEFCEEE54F0C4540F9018B693FF1200AC
:091856000EEE540F93FF02000E88
:10190200CDEFCDCCEECCEEFF121846CFEDCF0218C4
:01191200468E
:091980007BFF7A1879B30218EF1D
:0E0BCE008F468E458D448C438B478A4889495B
:100BDC00E4F553EC4D4E4F7017E94A4B70057F30DE
:100BEC0002000E1218C78F827583007430020CF14C
:100BFC001218D4EC33502AE5494548454770077F15
:100C0C002D12000E800D1218C78F82758300742D63
:100C1C0012069F1218D21207DE8F468E458D448C19
:100C2C0043755201754D00754CCA754B9A754A3B0C
:100C3C00E4FFFEFDFCAB4DAA4CA94BA84AD312080D
:100C4C00025003020CDC1218D2A84A12074C8F5126
:100C5C008E508D4F8C4EEC4D4E4F7004E5527023E0
:100C6C00E5512430FFE54945484547700512000E13
:100C7C00800EAE531218C98E82758300EF12069F38
:100C8C00E4F552AF4DAE4CAD4BAC4AAB51AA50A9AA
:100C9C004FA84E1206C1C8ECC8C9EDC9CAEECAC3EA
:100CAC00E5469FF546E5459AF545E54499F544E555
:100CBC004398F543AF4DAE4CAD4BAC4AE47B0AFACE
:100CCC00F9F812074C8F4D8E4C8D4B8C4A020C3C14
:100CDC00E548454945476010AB47AA48A9498553A3
:080CEC0082758300E412069FEB
:010CF40022DD
:10088B000134C35001DBBF68028BBB800344B798B4
:10089B000407B3B004D5AFC805A9ABE00689A7F828
:1008AB000775A410086DA02809719C400A819858FF
:1008BB000B9F94700CCA90880DE98CF90E048CA0D8
:1008CB000EA88AAC0F4D88B80FF786C410A184D040
:1008DB00115182DC120580E812BB7EF413747D008B
:1008EB0014307B0C14F2791815B8772416807530F8
:1008FB00174B733C1819714818ED6F5419C46D6080
:10090B001AA16B6C1B7E69781C6167841D4A65900C
:10091B001E37639C1F2561A8201A5FB421125DC08E
:10092B00220D5BCC230E59D8241557E4251F55F007
:10093B00262F53FC27425208285B501429764E2051
:10094B002A9B4C2C2BC04A382CEE48442E1E46506A
:10095B002F55445C308F426831D1407433173E8041
:10096B0034633C8C35B13A98370938A4386636B0C5
:10097B0039C734BC3B2D32C83C9D30D43E0F2EE0E2
:10098B003F882CEC41062AF8428D29044418271085
:10099B0045AB251C4741232848E121344A861F409B
:1009AB004C311D4C4DE21B584F9C1964515D177017
:1009BB005323157C54EF138856C4119458A20FA0DF
:1009CB005A830DAC5C6D0BB85E6009C4605807D0E0
:1009DB00625A05DC646203E8667301F4688A0000FE
:1009EB006AA1FE0C6CB8FC186ECFFA2470E6F830D6
:1009FB0000000000000000000000000000000000EC
:100A0B0000000000000000000000000000000000DB
:100A1B0000000000000000000000000000000000CB
:0C0A2B00000000000000000000000000BF
:1013CB0075F004E537A4248BF582E5F03408F5833A
:1013DB00E49322FE740193FF75F004E537A422F524
:1013EB0083C37401939FFFE4939EFEE4228F388E98
:0F13FB00378D368C35228F348E338D328C3122E4
:1018DB00C3EF9DEE9C400AD3EF9BEE9A50037F0122
:0418EB00227F002236
:040CF5008E358F3673
:100CF900E4F5371213CBFC740193FD1213E3248F2F
:100D0900F582E5F03408F583E493FA740193FBAFB7
:100D190036AE351218DBEF7003020DE51213CB1254
:100D290013DE248FF582E5F034081213EA8F3B8E27
:100D39003AF539F5381213E32491F582E5F03408D0
:100D4900F583E4931213DE248DF582E5F03408125D
:100D590013EA8F3F8E3EF53DF53CAD3DAC3C1207A5
:100D6900DE8F3F8E3E8D3D8C3CAE35AF36E4FCFDCB
:100D7900EEC0E0EFC0E01213CBFE740193FBCAEEA4
:100D8900CAD0E0FFD0E0FEC3EF9BFFEE9AFEED94E0
:100D990000FDEC9400FCAB3FAA3EA93DA83C12061D
:100DA900C1AB3BAA3AA939A838121346C8ECC8C93D
:100DB900EDC9CAEECACBEFCB1213E3248DF582E558
:100DC900F03408F583E493FE740193FFE4FCFDEB32
:100DD9002FFFEA3EFEED39FDEC38FC220537E537F9
:0D0DE900C3946A5003020CFCE4FFFEFDFC05
:010DF60022DA
:0100120022CB
:1011CE001213F8AB38AA37A936A835E8C0E078BDB7
:1011DE00E6FE08E6FFE4FCFDD0E0F81206C11213AD
:1011EE00F8780E1208131213F878BFE6FE08E6FF21
:1011FE00EE3395E0FDFCE5382FF538E5373EF53753
:10120E00E5363DF536E5353CF535AF38AE37AD361E
:02121E00FC22B0
:021271008D30BE
:10127300120CF51214011211CE121401E530146090
:101283001C14702DE47FE87E03FDFCAB34AA33A964
:1012930032A8311206C1E47BE87A0B800CAF34AE7E
:1012A30033AD32AC31E47B03FAF9F812134612146E
:0912B30001AF34AE33AD32AC31B1
:0112BC00220F
:10064700BB010689828A83E0225002E722BBFE02B1
:09065700E32289828A83E49322E4
:10066000BB010CE58229F582E5833AF583E022504F
:1006700006E92582F8E622BBFE06E92582F8E22299
:0D068000E58229F582E5833AF583E49322B3
:10068D00BB010689828A83F0225002F722BBFE014C
:02069D00F32246
:10069F00F8BB010DE58229F582E5833AF583E8F091
:1006AF00225006E92582C8F622BBFE05E92582C83D
:0206BF00F22225
:1006C100E88FF0A4CC8BF0A42CFCE98EF0A42CFCD8
:1006D1008AF0EDA42CFCEA8EF0A4CDA8F08BF0A456
:1006E1002DCC3825F0FDE98FF0A42CCD35F0FCEBB5
:1006F1008EF0A4FEA9F0EB8FF0A4CFC5F02ECD397A
:0F070100FEE43CFCEAA42DCE35F0FDE43CFC22E6
:1007100075F008758200EF2FFFEE33FECD33CDCCA0
:1007200033CCC58233C5829BED9AEC99E582984023
:100730000CF582EE9BFEED9AFDEC99FC0FD5F0D600
:10074000E4CEFBE4CDFAE4CCF9A88222B800C1B92A
:100750000059BA002DEC8BF084CFCECDFCE5F0CB68
:10076000F97818EF2FFFEE33FEED33FDEC33FCEBA1
:1007700033FB10D703994004EB99FB0FD8E5E4F95C
:10078000FA227818EF2FFFEE33FEED33FDEC33FC49
:10079000C933C910D7059BE99A4007EC9BFCE99A3D
:1007A000F90FD8E0E4C9FAE4CCFB2275F010EF2F82
:1007B000FFEE33FEED33FDCC33CCC833C810D70782
:1007C0009BEC9AE899400AED9BFDEC9AFCE899F8BD
:0E07D0000FD5F0DAE4CDFBE4CCFAE4C8F92250
:10134600C2D5E830E70FB2D5E4C39BFBE49AFAE4D2
:1013560099F9E498F8EC30E717B2D512137C120726
:101366004CE4C39BFBE49AFAE499F9E498F8800309
:1013760012074C30D50DE4C39FFFE49EFEE49DFDAD
:04138600E49CFC22C5
:0E07DE00C3E49FFFE49EFEE49DFDE49CFC222C
:1007EC00EB9FF5F0EA9E42F0E99D42F0EC6480C884
:0607FC0064809845F02224
:10080200EB9FF5F0EA9E42F0E99D42F0E89C45F04C
:0108120022C3
:10081300E86010ECA2E713FCED13FDEE13FEEF13FB
:04082300FFD8F022E8
:0C082700E6FC08E6FD08E6FE08E6FF22FD
:0D083300E6FB08E6F908E6FA08E6CBF82235
:0C084000ECF608EDF608EEF608EFF622E4
:10084C00D083D082E493F608740193F60874029373
:09085C00F608740393F6740473AA
:10086500D083D082F8E4937012740193700DA3A322
:1008750093F8740193F5828883E473740293686036
:06088500EFA3A3A380DF36
:00000001FF
